:10000000A8060020B9200000B5200000B52000009F
:1000100000000000000000000000000000000000E0
:10002000000000000000000000000000B5200000FB
:100030000000000000000000B5200000B520000016
:10004000B5200000B5200000990B0000B52000008D
:10005000390E0000B5200000B5200000B5200000DA
:10006000B5200000AD0D0000BD0D0000CD0D00005D
:10007000DD0D00000000000000000000B5200000C1
:10008000B5200000B5200000C1070000D107000026
:10009000E10700000000000000000000B5200000A3
:1000A000B5200000B5200000B5200000B5200000FC
:1000B0000000000010B5064C2378002B07D1054B3B
:1000C000002B02D0044800E000BF0123237010BDC4
:1000D0001800002000000000AC550000084B10B5CF
:1000E000002B03D00749084800E000BF0748036819
:1000F000002B00D110BD064B002BFBD09847F9E731
:10010000000000001C000020AC550000AC550000B1
:100110000000000070B50020084B98470500084C0F
:10012000FA218900A047074B186007492800A0471B
:10013000064B18600522064B1A6070BD151E0000A4
:10014000BD4E00000000002040420F0004000020CF
:1001500010E000E030B5084B1C68084A00258021FB
:100160004902013807D3002CFBD054609560136816
:100170000B42FCD0F5E730BD0400002010E000E0A9
:1001800030B5084B1C68084A002580214902013817
:1001900007D3002CFBD05460956013680B42FCD051
:1001A000F5E730BD0000002010E000E0044A1378BD
:1001B00002210B43137053785BB2002BFBDB7047BB
:1001C0000018004000B583B0124A936940210B43E8
:1001D000936101A900230B7005200F4B9847052060
:1001E0000E4B98470E4A137801210B431370537836
:1001F0005BB2002BFBDB0B4B19004031002204C328
:100200009942FCD11022084B1A60084B984703B062
:1002100000BDC046000400402D1F0000A11E0000CC
:10022000001800403C01002000E100E0AD010000AA
:100230000023036043600122027242728372023320
:10024000C3727047F0B583B005000C0001A900230C
:100250004B70CB7023790B70237A8B702078154B01
:10026000984700201F2D00D8134807222A409200EB
:10027000E77AA37A002B01D008231F43EB089B00E9
:10028000C31899690F269640B14397403A000A4334
:100290009A61637A002B06D143690122AA409343F5
:1002A000436103B0F0BD42690123AB401343436196
:1002B000F7E7C0465520000000180040F0B5CE46D4
:1002C000474680B583B005000C00160029600B6816
:1002D0001C209B0704D503B00CBC90469946F0BD8A
:1002E0000B681738DB07F6D40800494B9946984746
:1002F000484A116A831C0127B8469F403B000B43C4
:10030000136201A9737E0B701430C3B21F00180072
:10031000414B98473800414B9847707E0021404B35
:1003200098472868C84707003E493F4B9847BF0099
:100330003E4BFD5000232422AB540132AB54EB84DE
:10034000337E6B72102323602C683389EB80337CFF
:100350002B7280236A461370002353706B4642460B
:100360009A7000236A46D370F069356A002843D03A
:100370006B46187002236A465370000CC0B269467F
:100380002B4B9847002D3CD06B461D7002236A46CC
:1003900053702D0CE8B26946254B9847B37E8022F6
:1003A000002B04D1234B9B789B07DB0FDA012068DD
:1003B000736871690B432421715C89070B43252104
:1003C000715CC9060B432621715CC9050B430343CD
:1003D00013432360728980235B0013436360B389F6
:1003E0005B00F28952041343727C1343327CD203C4
:1003F0001343636200206EE7002120000E4B9847F4
:10040000B6E7012120000C4B98470500BCE7C04629
:10041000FD0C0000000400402D1F0000A11E000084
:10042000B50B0000B5040000490D00008C01002050
:100430005520000000200041010C00000123437200
:10044000704700234372704710B5931C9B00C3187C
:1004500059602424035D012191400B43DBB2035515
:1004600010BD028D0523002A01D0180070474B688B
:10047000C3620B8803850B88C38405323123C254C1
:10048000036802329A750023EFE7028D0523002AE4
:1004900001D0180070474B68C3620B8803850B8836
:1004A000C38405323123C254036802329A75002393
:1004B000EFE7000070B580008D4BC45825682523F8
:1004C000E65C2422A25C16402B7E9B0700D468E0E9
:1004D000637A002B2BD1E38C9BB2228D9A4200D100
:1004E000ECE03023E35C002B30D1B3072AD40023A7
:1004F0003122A354E38423856B8BDB0704D51022C0
:100500003123E254B30627D4637A002B00D1D9E01B
:100510006A688023DB0213436B606A68C0239B0216
:1005200013436B606B68734A13406B6070BD6A68FD
:100530008023DB0213436B606A68C0239B02134372
:100540006B60F3E7236920009847D0E7F307CED527
:10055000E36820009847CAE7236A20009847D3E75A
:10056000636920009847B7E06B68624A13406B608C
:10057000D3E700223023E254330709D4E38C9BB243
:10058000002B09D16A688023DB0213436B60C4E748
:10059000A36920009847F1E76B68564A13406B60E7
:1005A000BBE72B7EDB0730D500223123E2542C3B06
:1005B0002B752033E35C5B0705D42523E35C082B14
:1005C00001D002232B753123E35C1E2B12D0312383
:1005D000E35C102B0ED0B30703D53023E35C002B74
:1005E0000BD0F30703D53023E35C012B09D00023A4
:1005F000E384238501232B7698E72369200098471D
:10060000F5E7E36820009847F1E72B7E5B0700D40D
:100610008CE7238D002B1ED03022A25C012A13D040
:10062000E38C9BB2002B00D180E73023E35C002BEE
:1006300039D0E36A5A1CE2621B78DBB22822AB5441
:10064000238D013B238571E7E28C92B29342E7D27E
:100650006B8B5B07E4D53023E35C002B13D16A6816
:100660008023DB0213436B606A6880239B02134381
:100670006B601E223123E254F30600D456E7E3698F
:100680002000984752E76A688023DB0213436B60BF
:100690006A6880239B0213436B6000223123E2547B
:1006A0002D3B2B7542E7E26A531CE3622823EB5C87
:1006B000DBB21370238D013B238537E76B8BDB07A0
:1006C00000D51CE76B8B1B0700D452E701223023B7
:1006D000E254730700D543E7E38C9BB2002B00D0B4
:1006E00042E76A688023DB0213436B6015E7C0466C
:1006F0008C010020FFFFFBFF931C9B001950022A76
:1007000009D0032A0CD0012393401A00037E13431F
:10071000037600207047037E102213430376F8E728
:10072000037E202213430376F3E78B1C9B000022F9
:100730001A50022908D003290BD001228A40037ED7
:100740009343037600207047037E10329343037671
:10075000F8E7037E202293430376F3E770B5800029
:10076000164BC45823689D7B227E637E13401D4038
:10077000EB0706D4AB070BD4EB0610D4AB0615D4AD
:1007800070BD2000A3689847012322689373F1E7A6
:100790002000E3689847022322689373ECE7200067
:1007A00023699847102322689373E7E72000636961
:1007B0009847236820229A73E2E7C0467C01002014
:1007C00010B50020014B984710BDC0465D070000E2
:1007D00010B50120014B984710BDC0465D070000D1
:1007E00010B50220014B984710BDC0465D070000C0
:1007F00030B585B001AA0B4B32CB32C2019B984277
:100800000DD0029B984208D00023039A824202D066
:10081000180005B030BD023302E0012300E00023E0
:10082000DBB2F5E740500000F0B587B004000D00E2
:1008300016000800854B9847070005AB1B221A706D
:1008400001325A709A7003AB802212011A80802202
:1008500052015A80802292019A800023A360E360B3
:1008600023616361237663768200794BD4502560DF
:10087000B378082B06D023712B880520DB0705D51C
:1008800007B0F0BD1720FA07FAD5F4E7EB7B173075
:10089000DB06F5D42B889B07F2D4337C002B79D16F
:1008A000337F002B00D081E06A49086A7A0003ABED
:1008B000D35A03430B62B378082B00D186E001A919
:1008C00033780B7005ABDF5D3800634B9847380019
:1008D000624B98473189B3880B43B178B2791143A1
:1008E00019437378002B02D080231B01194322681F
:1008F000D37B5BB2002BFBDB2980717B4B1E9941C4
:100900008900B37B002B01D0012319432268D37BDC
:100910005BB2002BFBDBFF232B71002905D0226883
:10092000D37B5BB2002BFBDB6971B17AF37A002BCE
:1009300001D010231943337B002B01D0202319430E
:100940002268D37B5BB2002BFBDBA9712268D37BCF
:100950005BB2002BFBDB2379042B3FD0082B5ED04E
:100960001720002B00D08BE7D37B5BB2002BFBDB87
:10097000338D2B822268D37B5BB2002BFBDB738D24
:100980002B832268D37B5BB2002BFBDBB38D6B83A5
:10099000002075E702A901238B700022CA70327E05
:1009A0000A704B70307D2E4B984779E702A90123DE
:1009B0008B700022CA702432B21812780A704B7001
:1009C0001F33F3181878264B98476DE7086A7A1C8E
:1009D000520003ABD35A03430B6270E7D37B5BB285
:1009E000002BFBDB2823F35C2B742268D37B5BB2E8
:1009F000002BFBDB2923F35C2B752268D37B5BB2D6
:100A0000002BFBDB2A23F35C2B762268D37B5BB2C3
:100A1000002BFBDB2B23F35C6B76002030E7D37BD2
:100A20005BB2002BFBDBB36A2B612268D37B5BB22A
:100A3000002BFBDBF36AAB612268D37B5BB2002B3C
:100A4000FBDB336BEB6100201AE7C046F1070000C7
:100A50007C010020000400402D1F0000A11E0000AA
:100A6000552000000268D37B5BB2002BFBDB0379CF
:100A7000042B05D0082B0BD01720002B04D0704777
:100A8000C9B211740020FAE789B211820020F6E79A
:100A900011610020F3E7000010B582B00400394A6C
:100AA000936910210B439361374B1B785BB2102085
:100AB000002B03DBE3780730002B01D102B010BD1F
:100AC00022799A42FAD862799A42F7D82E4A137854
:100AD0000E398B431370D3795BB2002BFBDB637849
:100AE0000020002BEAD001A9A3780B700330274B1C
:100AF00098470320264B98472378002B27D1E3788B
:100B0000013B2279002A26D01F490A78042002439B
:100B10000A702279013A824013431B49CA7952B2C2
:100B2000002AFBDBDBB2184A53706379002B18D123
:100B30002378002B1FD0144A137880210B431370A5
:100B4000114AD3795BB2002BFBDB0020B6E7032010
:100B5000104B9847D3E70C490A78042082430A7067
:100B6000DBE71100CA7952B2002AFBDB013BDBB2A2
:100B7000054A9370DCE7044A137802210B43137093
:100B8000DEE7C04600040040001000402D1F0000BA
:100B9000A11E0000491F000010B50122034B9A71ED
:100BA000034B1B68002B00D0984710BD001000407D
:100BB0008801002010B582B004000E4B1B78002B7A
:100BC00007D0002905D10B4B5B78834210D01D2044
:100BD0000CE001A90C701320074B98471320074B1A
:100BE0009847044B5C7001221A70002002B010BDBF
:100BF0000020FBE7340000202D1F0000A11E000094
:100C00002B4B984223D00FD92A4B98422FD02A4BF6
:100C1000984242D101293AD0002946D0022938D041
:100C2000032938D0002039E0244B984235D10129DE
:100C300007D0002933D0022905D0032905D0002090
:100C40002CE01F482AE01F4828E01F4826E0012921
:100C500007D0002925D0022905D0032905D000207E
:100C60001CE01A481AE01A4818E01A4816E0012950
:100C700007D0002917D0022905D0032905D000206C
:100C80000CE015480AE0154808E0154806E015484C
:100C900004E0154802E0154800E0002070471448C1
:100CA000FCE70320FAE71348F8E71348F6E7C046E5
:100CB000000C0042001000420014004200080042F4
:100CC0000300050003000600030007000300010005
:100CD00003001E0003001F000300090003000A00B8
:100CE00003000B00030011000300120003001300B7
:100CF00003000400030008000300100030B585B0B5
:100D00006A460F4B32CB32C21B6813600300009A55
:100D1000824211D0019A82420AD0029A824209D0BC
:100D20000020039A9A4201D005B030BD033004E0A0
:100D3000012002E0022000E00020C0B2F4E7C0463B
:100D40004C5000007047000030B50B4B1B78002B57
:100D50000ED10A4C0A4D25600A4B00221A606560CC
:100D60005A60A5609A60E560DA600132024B1A7041
:100D70008000024BC15030BD3600002038000020FA
:100D8000450D00008C01002010B582B001AC092394
:100D90002370013363700133A3700133E370024B9E
:100DA0009847205602B010BDFD0C000010B5024B54
:100DB0001B680020984710BD3800002010B5024B7A
:100DC0005B680120984710BD3800002010B5024B29
:100DD0009B680220984710BD3800002010B5024BD8
:100DE000DB680320984710BD380000201723002A35
:100DF00001D0180070478B00064A9B58002B03D087
:100E0000834205D01D23F4E7890088500023F0E7D2
:100E10000023EEE73C0100201723002901D0180031
:100E2000704700221F2800D8024A01238340D36064
:100E30000023F4E70018004070B50022104B1A7030
:100E4000002310491F25104E0D4C0AE00D4908E003
:100E500023780133DBB223700F2B10D800211F2B16
:100E6000F4D9280018400122824008691042EFD0CE
:100E70000A619B009B59002BEAD09847E8E770BDB8
:100E80009C010020001800403C01002010B51F4AC2
:100E9000D36904210B43D3611D4B1A8B2021FF31F1
:100EA0000A431A831A7D0523D20701D4180010BD06
:100EB00003781B02C022920013404178C901FF222F
:100EC0000A401343817849001E220A401343C27826
:100ED00092048021C9020A40134302791204C021FE
:100EE00089020A4013430A4A536093685B035B0F0D
:100EF000084908249C400C8093684B8043780B7110
:100F0000138BDB05DB0F1B01D0E7C046000400405C
:100F1000004000414800002030B50400264A1088F7
:100F2000538843438B420BD280229201234BCB1830
:100F3000934205D9224A1820224BCB18934211D84C
:100F4000214B5D688022D2022A435A601A8B2020EE
:100F5000FF3002431A831B7DDB0704D41A4B5D600C
:100F60001B38FF3830BD452C22D8A300174AD35870
:100F70009F46154B1B8BDB0503D5134B5D60102083
:100F8000F0E789084900104BD96103E0890849005E
:100F90000D4BD961A520000204430B4B1C801900A6
:100FA00001220B7D1342FCD0074B5D600020D9E786
:100FB000054B5D601720D5E74800002000C07FFF8B
:100FC000FF0300000000C0FF004000415C50000033
:100FD000F8B5304B1C885B886343834207D22E4EA2
:100FE00018252E4BC318B34206D8012600E0002670
:100FF000631E1825184201D02800F8BD013D944217
:10100000FAD3274B1B7D123DDB07F5D5254C244B2E
:101010001C801D0001242B7D2342FCD0204C238BFF
:101020002025FF352B432383002A2CD001230500E4
:101030009D430023541EA44609E0CF187F783F0249
:101040003C432C8002339BB202359A4204D9CC5CDB
:101050006345F2DBA4B2F4E70E4B1B790025002BAD
:10106000CAD13F2AC8D8002E06D100220100042090
:101070000D4B98470500BFE7002201001C200A4BDA
:1010800098470500B8E7034B1B790025002BEAD0F1
:10109000B2E7C04648000020FF0300000000C0FF88
:1010A0000040004144A5FFFF190F000070B51C4B24
:1010B0001C885B886343834205D21A4E18251A4B5D
:1010C000C318B34203D8631E1825184201D0280064
:1010D00070BD013D9442FAD3144B1B7D123DDB07DA
:1010E000F5D5124C238B2025FF352B432383002A73
:1010F00014D0012398430023561E04E002339BB210
:1011000002309A4208D90488A4B2CC54B342F5DA2A
:10111000CD18240A6C70F1E70025D8E70025D6E742
:1011200048000020FF0300000000C0FF0040004115
:1011300010B51B4A138852885A43824207D2194C71
:10114000182219494118A14207D8012100E00021C5
:101150009B00013B1822184201D0100010BD134B18
:101160001B7D133ADB07F8D5104B1A8B2024FF3474
:1011700022431A8382085200DA6100290DD001232C
:101180009843002303800A4A084B1A801900012261
:101190000B7D1342FCD00022DFE7064AF4E7C0468D
:1011A00048000020FF0300000000C0FF0040004195
:1011B0001AA5000002A50000154B1A8B2021FF3153
:1011C0000A431A839B685903490F08228A40027018
:1011D00043801B0D83810F4B1B885B065B0F072B26
:1011E00010D00622D21A042393404360094B1B8877
:1011F00007221340072B08D00722D21A042393405A
:101200008360704700234360F0E700238360F8E7C2
:10121000004000410040800030B583B020490122E9
:101220000B7D1342FCD01F4B1B886A4613801E4B5C
:101230001B8853801D4B1B8893801D4B1B88D380BC
:10124000009B07221A4002705A06520F42709A04FD
:10125000920E82709A0B01210A40C270DA03920F3B
:101260000271019A140A0C4044715C0E0C408471A6
:101270009C0E0C40C4715C00240F047255000E24B7
:101280002C40DB0F2343437253061B0F8372D30999
:101290001940C172120C8281002003B030BDC046DB
:1012A0000040004100408000024080000440800077
:1012B00006408000F0B5DE4657464E464546E0B54E
:1012C00089B01723002821D041490C68414B1B6885
:1012D000019303789B4643789A468578C37899466C
:1012E000037902934379039383790493C379059334
:1012F000037A0693467A837A0793C37A9846878956
:1013000000220520344B9847031E07D0180009B06F
:101310003CBC90469946A246AB46F0BD00222C4903
:1013200044202D4B9847031EF0D1294907229443AE
:101330000733584603402343702083435446240117
:1013400020400343254C23402D02FC208001054012
:101350002B43234D2B40484685032B432148034014
:101360000298C00303432048034004984006034307
:101370001E4803400598800603431D480340069815
:10138000C00603435B005B08F00703430B60194B87
:101390000198184003000398000203439343760822
:1013A000334371329343079AD600334380229343E9
:1013B0004246D20113431B041B0C3F041F43054B41
:1013C0001F6000220620044B984703009EE7C0469A
:1013D0000040800004408000190F0000FFC0FFFFA4
:1013E000FFBFFFFFFF7FFEFFFFFFFFFDFFFFFFFBD4
:1013F000FFFFFF87FFFEFFFF00B583B001AB802238
:101400001A700A785A704A789A708A78DA701900D5
:10141000014B984703B000BD55200000F0B5234BA9
:101420001D89002D3DD058689F7A020000236E1E52
:1014300004E00133403299B2A9420CD29E42F8D066
:1014400011788CB2FF2CF4D0BC42F2D2174CA446D7
:101450006144CB72EDE73F218723144AD154AC0895
:1014600004220027002C14D11AE001339BB29342CE
:1014700007D09E42F9D09901095CFF29F5D00025DB
:10148000F3E7002D09D10137BFB2043292B2A7426F
:1014900006D0131F9BB20125EBE78723034AD754DD
:1014A000F0BD3F218723014AD154F9E750000020C5
:1014B000F8B50D008401054F054E7B6818194022D0
:1014C0002900B0470528F8D0F8BDC04650000020DC
:1014D000AD10000070B50402034E044D7368181976
:1014E000A8470528FAD070BD500000203111000037
:1014F000F8B50D008401054F054E7B681819402290
:101500002900B0470528F8D0F8BDC046500000209B
:10151000D10F000070B58401044E054D7368191990
:1015200000220420A8470528F8D070BD50000020F4
:10153000190F000010B59AB018AB002119700122E4
:101540005A702E4A5268D206120F9A70D9701971C9
:101550002B4C18A8A0470528FBD014A8294B984766
:10156000159B16200B2B01D81AB010BD264C2381D9
:101570001A00083A5208A2721B049B0A5B4280229E
:1015800012029446634463600022C823E2541F4B56
:1015900098478723E35C1A203F2BE5D001AA1C4B18
:1015A00013CB13C2184B1889013880B204A9194B08
:1015B0009847049B019A934219D1059B029A934242
:1015C00017D1069B039A934215D104ABDB7B102005
:1015D000012BC9D104AB1B7B012BC5D104AB5B7BB9
:1015E000002BC1D10122084B1A700020BCE71A2041
:1015F000BAE71A20B8E71A20B6E7C0460040004113
:101600008D0E0000B9110000500000201D140000D4
:1016100074510000B114000070B594B02F4C00223A
:101620008723E25400202E4B98472589042D25D985
:101630000026042419E0A008C0B2294B984704AD45
:101640004022FF212800274B98472E7029002000B8
:10165000254B98472000254B98470136B6B20134F8
:10166000A4B21E4B1D89A54208D9013DAC42F6D05B
:1016700003232340DFD0012BF1D8E0E701AE1C4B60
:10168000320013CB13C204AC4022FF212000154BC3
:101690009847019B049373686360B368A360012358
:1016A000E373237300236373A373013DEB170320DC
:1016B00018404519AD10E8B2094B9847074D2889E5
:1016C000013880B22100084B98472889013880B240
:1016D000064B9847074B984714B070BD5000002048
:1016E000D51400002F500000F11400001515000063
:1016F000745100001D14000010B590B00C00154B83
:101700001A781F23002A02D1180010B010BD114B07
:101710009A7A18238242F7D9B0330E4AD35C002B51
:1017200003D08823D35C83420CD00A4B1818C07AAC
:101730006946094B98473C2201A92000074B98476E
:101740000023E1E73C2203498C312000034B9847FA
:101750000023D9E750000020B11400001D50000004
:1017600010B5C823084AD35C002B01D1002010BD5E
:1017700014008823D35CD318D87A044B98470022EE
:10178000C823E254F2E7C0465000002015150000BF
:10179000F0B5DE4657464E464546E0B587B00400F4
:1017A00000915A4B1B781F20002B06D107B03CBC80
:1017B00090469946A246AB46F0BD544B9B7A0738FB
:1017C000A342F3D9C823514AD35C002B05D0882308
:1017D000D35CA34201D04E4B98474C4B1B19DE7A89
:1017E000032331009943494B5868B3011B5CFF2B1D
:1017F00047D0751CEDB20431C9B2A94257D06B1C59
:10180000DBB2AA01125CFF2A3CD01D00F5E705AA55
:10181000D218567069E005AFFF187D7063E07078EC
:1018200002993C4B9847394C21008831A8B23A4B79
:1018300098474B461B78E318DD720122C823E25417
:1018400001370236022F13D087235A46D55CAD00EC
:10185000ED19D047B146337801998B42DFD1882307
:101860002A4AD1543C22009903982C4B9847DAE736
:10187000444640462A4B98478723244AD4540020A4
:1018800094E73500214E8823F45430008C303C22FC
:101890000099224B984731008831A8B21E4B9847D7
:1018A0003419E5720122C823F25400207EE7B30800
:1018B00098461B02154A5268D31805AA1978117068
:1018C00003218E4356703D31595C9170711CD1706B
:1018D0008022985C4032995C0023B51C033605AA2F
:1018E000D25C904297D08A4291D00233042BF6D139
:1018F00005AE0027054B9B46054B9A465B46883351
:1019000002930433039301949EE7C04650000020E5
:1019100061170000B1140000F11400001D50000018
:10192000D5140000704700000C4B1B68002B06D13B
:10193000EFF31083002B07D00022094B1A70074ADF
:10194000136801331360704772B6BFF35F8F0022D4
:10195000044B1A700132024B1A70F0E71C01002090
:101960002001002008000020084B1A68013A1A6084
:101970001B68002B09D1064B1B78002B05D00122D8
:10198000044B1A70BFF35F8F62B670471C010020D2
:10199000200100200800002010B5082803D880008E
:1019A0001B4B1B589F46002030E01A4B18692DE056
:1019B000194B1B6A9B059B0F1848D84026E0154B16
:1019C000586923E0134B1B6800209B071ED5124962
:1019D0001022CB681A42FCD00E4B1B685B0701D467
:1019E0000F4813E000200F4B98470A4B9B681B04DD
:1019F0001B0C58430AE05023074AD35C00205B07C6
:101A000004D5044BD86801E08020000210BDC04618
:101A100080510000240100200008004000127A00DC
:101A2000006CDC02791F000070B50C490B6A047869
:101A3000857840780122104080014026B34303435B
:101A40002A40D20180208343134303222240120202
:101A50000348034013430B6270BDC04600080040BA
:101A6000FFFCFFFF10B5037A9B061B0C4289920511
:101A7000920D134318494B608379C279134342880E
:101A80008488224313434278D20113430B600378C6
:101A9000042B11D0202B0ED1037B9B06028A13430B
:101AA000C28912040D490A4013430B4A936011681E
:101AB0000B4B0B43136010BD037B9B06028A134341
:101AC000C289120405490A401343034A936013680C
:101AD00004210B431360EEE7240100200000FF0304
:101AE00024040000082803D88000254B1B589F467B
:101AF000172044E0234A136A02210B43136200209B
:101B00003DE0204A936902210B439361002036E0B7
:101B10001C4A138A02210B43138200202FE0194A2A
:101B2000938A02210B439382002028E016490B6818
:101B3000022213430B60134B9A8419000E32CB68B8
:101B40001A42FCD0104A91680E4BD96252689A62D0
:101B500000229A8419001032CB681A42FCD00A4B3A
:101B60001B689BB2074A9384002008E00549442281
:101B70008B5C022003438B54002000E00020704760
:101B8000A45100000008004024010020082832D899
:101B900080001A4B1B589F46194A136A02218B4337
:101BA000136200207047164A936902218B439361A8
:101BB0000020F7E7124A138A02218B431382002088
:101BC000F0E70F4A938A02218B4393820020E9E7D2
:101BD0000C4B1A6802218A431A601B689BB2084AA0
:101BE00093840020DEE7064944228B5C0220834375
:101BF0008B540020D6E71720D4E7C046C851000018
:101C00000008004024010020082805D88000114B5E
:101C10001B589F46042312E0002017E002230EE029
:101C200010230CE050230C4AD05C4D3B1840033885
:101C300043425841C0B209E0082300E00123064AAC
:101C4000D0681840C01A43425841C0B270470120C2
:101C5000FCE7C046EC5100000008004030B585B0FC
:101C6000C222D2001A4B9A601A4A53681E218B4333
:101C7000536001236A4613700024174DE0B2694691
:101C8000A8470134252CF9D103A80024447001256C
:101C900085700470114B98470620114B9847114BE3
:101CA0009847114B1C725C729C72DC7201956B46FA
:101CB0005C7006236A4613701472547269460020E1
:101CC0000A4B984700200A4B984705B030BDC046E4
:101CD00000080040004000412D1F0000291A0000AC
:101CE000E51A0000F51C000000040040191D00006A
:101CF000D11D0000064A936908210B43936101221C
:101D0000044B1A7019000B781342FCD17047C0467F
:101D100000040040000C004070B5060004000D787F
:101D20002D0205434B78002B02D08023DB021D439C
:101D30004B7A002B02D080231B031D4348680128E7
:101D400010D9431E184234D1022830D90223002270
:101D500001325B009842FBD8120232431400802308
:101D60005B031D430B7A002B02D080239B031D4392
:101D7000134A53785BB2002BFBDB124B9847124B94
:101D80001E700F4A53785BB2002BFBDB0C4B9C6040
:101D90001A0053785BB2002BFBDB094A53688021A1
:101DA00049020B401D435560084B984770BD002207
:101DB000D2E70402344380239B021D43D2E7C0468E
:101DC000000C004029190000080C004069190000AF
:101DD00010B504000B4A53785BB2002BFBDB0A4BB7
:101DE00098470A4B1C70074A53785BB2002BFBDB09
:101DF000044A516880235B020B435360044B9847AD
:101E000010BDC046000C004029190000040C004021
:101E10006919000070B504001A4A53785BB2002BB0
:101E2000FBDB194B9847194B1C70164A53785BB271
:101E3000002BFBDB134E7068C004C00E144B984798
:101E40000500124B1C707668F602F60F114B1C70E1
:101E50000C4A53785BB2002BFBDB0A4B9C682402D4
:101E6000240C0D4B9847002E07D1012C07D92100D7
:101E700028000A4B9847050001E00134E54028009E
:101E800070BDC046000C004029190000040C004041
:101E900099190000080C004069190000BD4E0000AF
:101EA00010B50400064B9847064B1C70064A538831
:101EB0008021C9010B435380044B984710BDC04695
:101EC00029190000020C0040000C004069190000B4
:101ED00010B504000F4B98470F4B1C700F4A5388E6
:101EE0001B05180F53880E490B40538053880D492A
:101EF0000B40538011008022D2014B881342FCD149
:101F000006494A8803020648024013434B80064BA9
:101F1000984710BD29190000020C0040000C004039
:101F2000FFF0FFFFFFBFFFFF6919000010B50C783D
:101F300024020443024B9847A4B2024B5C8010BDBC
:101F4000D11E0000000C004010B50400064B98475D
:101F5000064B1C70064A5388802109020B435380AC
:101F6000044B984710BDC04629190000020C0040E0
:101F7000000C00406919000010B50400064B98479A
:101F8000064B1C70064B5C882405240F054B9847B4
:101F90002000054B984710BD29190000020C004095
:101FA000000C004069190000151E000030B5D37800
:101FB000002B35D11378802B29D01B068024640296
:101FC000234354780225AC4306D19478002C20D1C9
:101FD0008024A402234341605478013C012C1CD985
:101FE0000D042D0CA024E4052C431C4384620D0C2D
:101FF000D02424062C431C438462D478002C22D1A4
:102000005B031CD59378012B1ED0416117E00023A0
:10201000D7E7C024E4022343DDE70D4C2340DFE78C
:1020200041600C04240CA023DB05234383620C0CC9
:10203000D0231B0623438362D378002B03D153782C
:10204000013B012B02D930BD8161F8E78160FAE7DD
:10205000FFFFFBFF10B50A00C1090023002904D1CE
:102060004309DB0105498C4663441F2420400121BC
:1020700081401800024B984710BDC0460044004103
:10208000AD1F00007047000010B5054B9847054B89
:102090009847054B9847054B9847054B984710BD07
:1020A0005D1C00002519000085200000C50100000E
:1020B00085200000FEE70000F8B52A4A2A4B9A4224
:1020C00011D01A00294B9A420DD2294A03339B1A88
:1020D0009B0801339B000022234822498C588450DE
:1020E00004329A42FAD1234A234B9A420AD2D3436A
:1020F00021495B1803218B4304339B18002102C242
:102100009342FCD11D4AFF211D4B8B439360FD3947
:1021100090235B001B4AD1501B4AD3780325AB4365
:1021200002242343D370D3780C27BB4308263343C0
:10213000D370164B987B3022904320221043987323
:10214000997BB943314399739A7BAA4322439A738B
:102150000F4A536880210B4353600E4B98470E4B38
:102160009847FEE7AC550000000000201800002052
:102170000400002018000020A802002000ED00E06C
:102180000000000000700041005000410048004184
:1021900000400041D54F0000E93400000C4B1A68A4
:1021A000D37B5BB2002BFBDB8023537109490B68A7
:1021B00001330B60D37B5BB2002BFBDB002313717D
:1021C000D37B5BB2002BFBDB402353717047C046CF
:1021D000B4010020D80100200C4B1A68D37B5BB2FD
:1021E000002BFBDB8023537109490B6801330B6023
:1021F000D37B5BB2002BFBDB00231371D37B5BB281
:10220000002BFBDB402353717047C0466002002067
:1022100040020020022302009A43012A03D0023820
:1022200001281BD970471B4B1A68D37B5BB2002B6C
:10223000FBDB802353710021174B1960D37B5BB20A
:10224000002BFBDB00231371D37B5BB2002BFBDB8A
:10225000402353710122114B1A70E0E7104B1A68AA
:10226000D37B5BB2002BFBDB8023537100210D4B32
:102270001960D37B5BB2002BFBDB00231371D37B94
:102280005BB2002BFBDB402353710122064B1A701B
:10229000C8E7C046B4010020D80100201402002085
:1022A0006002002040020020A50100202C4B1B787A
:1022B0009B069B0F012B0CD0294B1B789B069B0F79
:1022C000022B18D0264B1B789B069B0F032B24D088
:1022D0007047244B1B78DBB2D9090022002904D1B6
:1022E0005A09D20120498C4662441F21194001231A
:1022F0008B405361ECE71D4B1B78DBB2D909002200
:10230000002904D15A09D20117498C4662441F2181
:10231000194001238B405361DAE7124B1B78DBB283
:10232000D9090022002904D15A09D2010E498C464C
:1023300062441F21194001238B4053610B4B1B78D2
:10234000DBB2D9090022002904D15A09D201064979
:102350008C4662441F21194001238B405361B7E72B
:10236000B00100201A020020004400415802002061
:10237000012848D0032809D0002810D0831E012B43
:1023800040D8234B1B78002B2CD020E0214B1B780E
:10239000002B08D11E4B1B78002B18D132E01D4BAF
:1023A0001B78002B0FD000221A4B1A701A4B1A6898
:1023B000D37B5BB2002BFBDB80235371831E012B8D
:1023C000DFD900281ED1124B1B78002B0CD0002225
:1023D0000F4B1A70114B1A68D37B5BB2002BFBDBDF
:1023E0008023537100280DD10D4B1B781B079B0FC9
:1023F000012B07D00B4B1A68D37B5BB2002BFBDBA6
:10240000802353717047034B1B78002BFAD0CAE727
:10241000A501002014020020B40100206002002069
:10242000B00100201C02002010B500230385064BDC
:10243000064A52689A4203D00120054B984710BDC6
:1024400000221A70F8E7C0469902002048020020D6
:1024500055010000F0B5D64600B584B0009001915A
:102460001500DA090027002A04D15F09FF01214A7B
:10247000944667441F22134001269E403B6A334026
:102480005A1E9341DBB203AA1370009A9A422ED0CF
:10249000FA239B00019A5A43924601240FE00198C7
:1024A000154B984702E05046144B98473B6A33401F
:1024B0005A1E934103AAA3540134032C07D0012DC3
:1024C000EDD0022DEFD001980C4B9847EEE71300AA
:1024D00052781B78934204D0009804B004BC924612
:1024E000F0BD03AB9B789A42F6D10093F4E70093DA
:1024F000F2E7C046004400415501000081010000A0
:1025000010B50523012205210120024CA047024BF2
:10251000187010BD552400001B02002000B587B0C4
:1025200001A8002202700023428082808371C3715F
:1025300007320272383242813E3A0273C28105325A
:1025400002824370054B9847054A53681E218B430E
:102550001A390B43536007B000BDC046651A00002E
:102560000040004100B585B001AB0122029200227B
:102570005A70062119701A725A7200280AD104235F
:10258000029301A90020054B98470020044B98476F
:1025900005B000BD07321A70F3E7C046191D0000F0
:1025A000D11D000010B590B0040001A900202E4BF1
:1025B0009847002C52D101ABB0221A7130325A71B7
:1025C00000221A735A739A73DA7301ABE2221A74F7
:1025D000DE3A5A74C0329A74BB3ADA74882119759B
:1025E0000A325A75102098751730D87519765A76B0
:1025F0003D329A767332DA7601AB19794908302286
:1026000052420A431A702120684400221978521855
:1026100092B201339842F9D101AC52426277210063
:102620000020124B9847124B9847210001200E4B77
:102630009847104B1B78002B0BD10021302301AAA7
:10264000D15401A90120094B9847094B984710B074
:1026500010BDFF21302301AAD154F2E7064B1B78AD
:102660009B06C9D5B1E7C046F916000091170000D6
:1026700061170000DD010020A401002010B504490D
:1026800009230B80034B4B60034B984710BDC0469A
:1026900050020020800200206304000000B583B0D7
:1026A000FF226B46DA71464B1A78B42A00D980E0D3
:1026B0009300444AD3589F46434B01221A80434A11
:1026C0005A604149424B984703B000BD3E4B01223E
:1026D0001A80404A5A60F4E73B4B01221A803E4A76
:1026E0005A60EEE7384B01221A803C4A5A60E8E70C
:1026F000354B01221A803A4A5A60E2E7324B0122F6
:102700001A80384A5A60DCE72F4B01221A80364A79
:102710005A60D6E72C4B01221A80344A5A60D0E71F
:10272000294B04221A80324A5A60CAE7264B0422F7
:102730001A80304A5A60C4E7234B04221A802E4A7A
:102740005A60BEE7204B04221A802C4A5A60B8E730
:102750001D4B01221A802A4A5A60B2E71A4B022204
:102760001A80284A5A60ACE7174B06221A80264A7C
:102770005A60A6E7144A04231380234B06335360A0
:102780009FE7114B04221A80204A5A6099E70E4BAA
:1027900001221A801E4A5A6093E70B4B08221A80C6
:1027A0001C4A5A608DE7084B01221A801A4A5A6067
:1027B00087E7054B01221A806A4607325A6080E794
:1027C000A00100201052000048020020DC0100207F
:1027D0008B0400005C02002044020020B0010020B5
:1027E000A40100209C020020A402002098020020E6
:1027F000940200207C020020D0010020A8010020CB
:102800003C020020180200200C000020A002002042
:10281000590200208C0200209A02002010B52F4B94
:102820001B789B069B0F012B10D02C4B1B789B0613
:102830009B0F022B1CD0294B1B789B069B0F032B55
:1028400028D000212648274B984710BD264B1B78DF
:10285000DBB2D9090022002904D15A09D201234947
:102860008C4662441F21194001238B409361E8E7A5
:102870001F4B1B78DBB2D9090022002904D15A0969
:10288000D2011A498C4662441F21194001238B4012
:102890009361D6E7144B1B78DBB2D90900220029DB
:1028A00004D15A09D20111498C4662441F211940B2
:1028B00001238B4093610E4B1B78DBB2D9090022B8
:1028C000002904D15A09D20108498C4662441F21CB
:1028D000194001238B409361B3E7C046B00100204B
:1028E0001C020020650A00001A020020004400417A
:1028F0005802002010B590B001225D4B9A6101286A
:1029000036D000281BD002284CD0032864D00024E5
:10291000584B1B78002B00D07EE00120564B984787
:10292000564A1368022BFCD90120554B9847002CBE
:1029300000D07CE00122534B1A7010B010BD5249F8
:102940000B789B079B0F01330A7803201840032361
:102950009A43130003430B704C4B1B78DBB2FF2BE5
:1029600052D04A4A13780133DBB213700124CFE707
:10297000454803781B079B0F013302780321194058
:1029800089000C239A4313000B4303703F4B5B7881
:10299000DBB2FF2B3AD03D4A53780133DBB25370A0
:1029A0000124B5E7384803789B069B0F0133027872
:1029B00003211940090130239A4313000B4303708C
:1029C000324B9B78DBB2FF2B22D0304A9378013315
:1029D000DBB2937001249BE72B490A789209531CC0
:1029E00003221A40087892013F23034013430B70DF
:1029F000264BDB78DBB2FF2B0CD0244AD378013393
:102A0000DBB2D370012483E7002481E700247FE751
:102A100000247DE700247BE70220174B98471C4ADF
:102A20001368022BFCD90220154B98477FE701ACB5
:102A300021000020174B9847144B1A7822735A78BC
:102A400062739A78A273DB78E373212068440023D1
:102A500022789B189BB20134A042F9D101A95B42B4
:102A60004B7700200C4B98470C4B984762E7C046C9
:102A7000004400411402002015220000D80100206B
:102A8000712300009B0200203C02002094020020E1
:102A900040020020F91600009117000061170000A5
:102AA000F0B5CE46474680B58FB0002823D1534BB2
:102AB0001A68D37B5BB2002BFBDB802353711021A0
:102AC00011734E4C637E8B4363760E3920004C4D60
:102AD000A847202223681A73637E934363760321F9
:102AE0002000A8472268D37B5BB2002BFBDB138856
:102AF00002218B43138001AB00229A7000219A803F
:102B000099711A8159709972D972197399731974DC
:102B10005A619A6119771A625A621A855A859A859A
:102B200001321A705A73374B1B781B079B0F51D118
:102B3000354A118801AB598552889A852F4D334CFF
:102B400001AA33492800A0470028F9D12B4B1A6865
:102B5000D37B5BB2002BFBDB138802210B4313807A
:102B6000264B1A68D37B5BB2002BFBDB80235371AF
:102B7000224C022227492000274DA847032227493B
:102B80002000A8472068264B99469847254B984631
:102B90001B5C1F26334001252A009A40224F3A60D1
:102BA000637E102213436376102322685373100050
:102BB000C84743461B5C1E40B5403D60637E2022F3
:102BC00013436376236820225A730FB00CBC9046DF
:102BD0009946F0BD0B4B1B781B079B0F032B06D0B0
:102BE000124A118801AB598552889A85A6E7104A86
:102BF000118801AB598552889A859FE71C020020F5
:102C00002B070000B0010020A801002029080000C7
:102C1000002C0042AD220000F90600001D28000033
:102C2000F10700008855000000E100E0D00100201D
:102C30007C02002010B55F4B1A68D37B5BB2002B7F
:102C4000FBDB802353715C4B1B789B069B0F012B96
:102C500046D0594B1B789B069B0F022B63D0564BDB
:102C60001B789B069B0F032B00D17FE0534B1B78F7
:102C7000DBB2D9090022002904D15A09D2015049F6
:102C80008C4662441F21194001238B4053614D4BF8
:102C90001B78DBB2D9090022002904D15A09D201DC
:102CA00047498C4662441F21194001238B405361E0
:102CB000414B1B781B079B0F012B10D00020424B70
:102CC00098473C4B1A68D37B5BB2002BFBDB00239D
:102CD0001371D37B5BB2002BFBDB4023537110BD20
:102CE000364B1B78DBB2D9090022002904D15A09DE
:102CF000D20133498C4662441F21194001238B4085
:102D00009361304B1B78DBB2D9090022002904D132
:102D10005A09D2012A498C4662441F2119400123D5
:102D20008B405361C4E7254B1B78DBB2D9090022E5
:102D3000002904D15A09D20121498C4662441F213D
:102D4000194001238B4053611E4B1B78DBB2D9091C
:102D50000022002904D15A09D20119498C46624443
:102D60001F21194001238B409361A1E7134B1B786E
:102D7000DBB2D9090022002904D15A09D201104935
:102D80008C4662441F21194001238B4093610D4BF7
:102D90001B78DBB2D9090022002904D15A09D201DB
:102DA00007498C4662441F21194001238B409361DF
:102DB0007EE7C0461C020020B00100201A0200205D
:102DC0000044004158020020A12A000030B591B013
:102DD0000400C38C9BB2028D9A4209D0BB4B1A7877
:102DE000BB4B1A703123E35C002B05D011B030BD12
:102DF000FF22B74B1A70F5E72000B64B9847E28CDC
:102E000092B2218D8A4210D0E38C013B5B1AB24A08
:102E1000138001A90020B14B9847AD4B1A78282A9E
:102E200058D89300AE4AD3589F460022AA4B1A8026
:102E3000EFE7A94B1B88012B4CD1A44B5B784022B8
:102E400052421A43131CA7490978C90746D4A54A18
:102E5000127892074AD4A34A127852074DD4A14A55
:102E60001278120750D49F4A1278D2064FD49E4A45
:102E70001370137801AA1278D0210B439A424DD0D7
:102E8000994B1B7830225242134301AA1370CF3959
:102E90000122964B1A7000291CD001AA21206844F7
:102EA000002311785B189BB201329042F9D101A93D
:102EB0005B424B7700208E4B98478E4B9847844B54
:102EC0001B78002B06D1884B1B789B079B0F022B8E
:102ED00000D15EE12000884B984787E7824B1B7842
:102EE0009B079B0F03218A431343B0E77E4A127866
:102EF00004210A408B431343ADE77B4A1278082133
:102F00000A408B431343AAE710221343ABE7764AE8
:102F1000127820210A408B431343A8E70021B7E72A
:102F20006D4B1B88012BD5D1684B5B7880221343F6
:102F3000724A137001226D4B1A70CBE7664B1B88E7
:102F4000012BC7D1614B5B78032213436C4A13708A
:102F50006C4B9847BEE7604B1B88012BBAD15B4B8B
:102F60005B7880221343684A13701378DBB201AA9E
:102F700012799A4224D0644B1A7801AB1A7101215C
:102F8000614B1B785B08D0221343574A13701378A8
:102F9000DBB201AA12789A4204D0534B1A7801ABE3
:102FA0001A7001210122514B1A70574B1B78DB0715
:102FB00008D41022554B1A700132554B1A706AE72B
:102FC0000021DDE71032514B1A70013A504B1A7054
:102FD00061E7414B1B88012B00D07BE73B4B5B78C3
:102FE000E02213433F4A13701378DBB201AA5279EF
:102FF0009A4200D16EE73B4B1A7801AB5A714CE70D
:10300000354B1B88012B00D064E7304A5378FE21F2
:103010000B435370FE2B03D00122344B1A7059E737
:10302000FF223C4B1A70F7E72B4B1B88042B00D078
:1030300050E7264A93781B0251780B43D178090454
:10304000354803400B43127912061B021B0A134337
:103050009AB2190C914200D83CE730498A4200D814
:1030600038E72F4A1360117801AB197451785974FD
:1030700091789974D278DA740FE7174B1B88042B78
:1030800000D027E7114A93781B0251780B43D1787F
:103090000904214803400B43127912061B021B0A44
:1030A00013439AB2190C914200D813E71B498A4284
:1030B00000D80FE71B4A1360117801AB19755178DE
:1030C000597591789975D278DA75E6E68002002014
:1030D000A00100203D04000046020020F916000077
:1030E000E45400009C020020DC0100201B020020B0
:1030F0009117000061170000430400005C020020EB
:10310000B0010020352C0000A40100201A0200208C
:103110005802002098020020FFFF00FFE703000094
:103120007C020020D0010020214B1B88042B00D002
:10313000D0E6204A93781B0251780B43D1780904DA
:103140001D4803400B43127912061B021B0A13434E
:103150009AB2190C914200D8BCE618498A4200D8AC
:10316000B8E6174A1360117801AB19765178597691
:1031700091789976D278DA768FE60D4B1B88022B00
:1031800000D0A7E60B4A51780E4B197092785A700E
:10319000A0E601AD290001200B4B9847FF22302308
:1031A000EA5429000120094B9847094B984791E6BA
:1031B0004602002080020020FFFF00FFE70300001E
:1031C000A801002018020020F91600009117000045
:1031D00061170000F0B5D646474680B593B08046EB
:1031E0000E001700AC490B78012293430B70AB4BD8
:1031F0001A700220AA4B9847AA4B1B785B075B0FFB
:10320000072B70D0FF22A84B1A700124002F06D084
:10321000A64B80225A618022D2015A610024002EDE
:1032200067D08022D202A14B9A614346002B65D021
:10323000802212039D4B9A61002E2CD0964B1B7856
:103240009B0660D4DE22944B1A700120984B98475D
:1032500003AD29000020974B98472A78964B1A70A7
:10326000EA7C964BDA70AA7C9A706A7C5A702A7C47
:103270001A70EA7D924BDA70AA7D9A706A7D5A7054
:103280002A7D1A70EA7E8F4BDA70AA7E9A706A7E67
:103290005A702A7E1A708C4B1B789B09022B0DD01A
:1032A0004346002B00D1E4E0874B1B787B2B00D1F9
:1032B000EDE07B22844B1A70844B98470220844BAC
:1032C0009847002F54D180225200784B5A61012C2C
:1032D00045D1804B1B68222B41D800239A467E4B58
:1032E00098467C4E27E0704A1378013BDBB213709E
:1032F0008BE78022D2026D4B5A6196E7802212033F
:103300006A4B5A6198E7FE22634B1A709DE76E4B39
:103310001B785B2BD2D05B226B4B1A706B4B9847A0
:10332000CCE780225200614B9A610137002D15D005
:103330003368222B13D80F2301220A210120C04712
:103340000500002FF2D1FA204000644B984701237A
:103350009C46E2445346512BE8DDE2E70024534B00
:10336000802252009A61803A5A618022D2015A61C9
:10337000002C11D1574B1B68222B0DD8564D554EA2
:103380000F2301220A210020A847002803D1336817
:10339000222BF5D900E001244E4B1B68222B15D8B7
:1033A00016254D4E4E4F4B4B984620000F230122C1
:1033B0000A21B047002823D00520B847013D002D41
:1033C00004D043461B680124222BEED90220344B43
:1033D0009847364B8022D2019A6180229A613D4BF8
:1033E0001B68222B38D80220394B98472A4B1B7870
:1033F00003209B0637D513B00CBC90469A46F0BD0F
:10340000012501270024334B9A46334E53461B684F
:10341000222BDBD8781E8741F8B21C2301220A2117
:10342000B047070000906B1E9D41E8B21B230122AC
:103430000A21B04705000190601E8441E0B20F23CD
:1034400001220A21B047041EE0D0009B002BDDD0F2
:10345000019B002BDAD0B9E70320224B98470E4B93
:103460001B780120C7E70C4A137840218B43137067
:10347000C1E7002E00D14AE7134B1B785F2B00D128
:103480001CE75F22104B1A70104B984716E7002E6E
:1034900000D113E7F0E7C0465C0200201B020020C9
:1034A0007123000044020020A402002000440041D7
:1034B000A5250000F9160000DC0100207C02002098
:1034C000D0010020A8010020B0010020352C000010
:1034D0001522000040020020552400005501000084
:1034E00081010000F5280000F0B5DE4657464E4643
:1034F0004546E0B5AFB0FF22AC4B1A700021002367
:10350000AB480170AB480180AB4900200870FE2039
:10351000AA4908703E38AA490870AA490A70AA49FF
:103520000B70AA490A70F021A94A1180A94A1370A8
:10353000A94A1370A94A1370A94A1370A94A1370B3
:10354000A94A13700122A94B1A70A94B9847A94B9D
:1035500098470720A84B9847002804D0A64C07207E
:10356000A0470028FBD10120A44B984710AC0025B0
:1035700065700623237025726572C8239B00636003
:10358000210001209E4B984701209E4B9847012621
:10359000267021001B209C4B984698471B209B4F70
:1035A000B84721001C20C0471C20B84721001C2020
:1035B000C0471C20B847964B1E70BFF35F8F62B6A2
:1035C000944B98470020944FB847944B1B7ADBB23A
:1035D000D840934B18600120B847924B18600CAB51
:1035E0001D705E70904B5B68DB061B0F0CAA93701E
:1035F000D570157110008D4B984720008C4B984763
:103600006378032B03D110ABDB79002B17D010A804
:1036100003234370113383700024C47004710125A7
:1036200045718471C471834B98470EA8047045702E
:103630000471447184700423C3707F4B98477A49A6
:1036400001220B7D1342FCD07C4B1A687C4B1A6024
:103650007C4A12685A603823704AD35CDBB27A4ADB
:1036600013701278544B1A7010AC00262670042385
:103670009946A3700C23E370267166716670200072
:103680006D4B98472670A6706670210006206F4D1E
:10369000A84721000920A84721000420A8472100AD
:1036A0000520A84721000A20A84721000B20A84791
:1036B00021000F20A84721001820A8472100012041
:1036C000A84721001920A84721001B20A847210056
:1036D0001C20A847012398466370A6700227277014
:1036E00021000220A84721000320A847210007202D
:1036F000A84721000820A84721000E20A847210044
:103700001220A84721001320A84721000020A84725
:1037100021001020A84721001120A8474C4B4A4601
:103720009A6104325A6178325A6180325A61802239
:10373000D2015A618022D2025A61802212035A6158
:1037400042465A61802252025A61802292025A6194
:103750002000404B984705231093A023DB026360B1
:103760002672E772210005203B4B98470022052175
:103770003A483B4B9847002105203A4B98473A4B33
:1037800098476423162800D17CE0002872D12E4B84
:103790001A780023402A75D1344A117820330B431C
:1037A00013700120324B9847C8236BE0A001002022
:1037B00099020020460200209A0200205C020020AC
:1037C00044020020980200203C020020A4020020B5
:1037D00018020020DD0100209B020020AC01002027
:1037E0005D02002014020020A50100201B02002021
:1037F000892000001D250000E51A00006525000055
:10380000191D0000D11D00002D1F0000A11E000089
:103810000800002015010000151E000000040040F3
:10382000A0020020D4010020004000418D0E0000C5
:1038300019120000B5120000990A00000040800033
:103840008C0200200440800038020020F9130000A0
:103850000044004131020000450200000125000043
:10386000ED0D0000190E000035150000A401002028
:10387000A5250000D24B9847D24B98470020D24B49
:103880009847C823D14A13701FA90020D04B9847EE
:103890001FA96A200CAB9C46604400230A789B1841
:1038A0009BB201318142F9D1DBB2002B0BD0C94A66
:1038B000137820210B4313700120C34B98471FA995
:1038C0000020C34B98471FAB1978C34A11701A796F
:1038D000C0490A705879C14A1070D87CC04AD0706B
:1038E000987C9070587C5070187C1070D87DBD4AC0
:1038F000D070987D9070587D5070187D1070D87E73
:10390000B94AD070987E9070587E5070187E1070B2
:10391000D87BB64AD070987B9070587B50701B7BD8
:1039200013700B78DB0700D443E11122B04B1A70FF
:10393000013AB04B1A7010AA0021117080239B032A
:10394000536001235B42138100235181D1811374A1
:103950005374516113765376937624315354013165
:1039600053540131535458239381A34BD361A34B38
:103970001362A349A348A44B9847002813D1A14D33
:103980002C682000A14B98471F2318401E3B834002
:103990009F4A13602A680323D1690B42FCD1236834
:1039A000022213432360974C02229A4920009A4D29
:1039B000A847032299492000A847002298492000DF
:1039C000A847012297492000A8472523E25C04214B
:1039D0000A43E254216802208875E25C08252A43E4
:1039E000E2548875E25C013801210A43E254E25C4A
:1039F00001310A43E25410AB002200219A709A71FF
:103A00001A8100245C709972D972197399731974B0
:103A10005A619A6119771A625A621A859A851870E2
:103A20008022D2009A80804A5A8558737F4D804CFC
:103A300010AA80492800A0470028F9D17B4B1A68BA
:103A4000D37B5BB2002BFBDB138802210B4313807B
:103A5000764B1A68D37B5BB2002BFBDB8023537160
:103A600010AB002200219A709A711A8100205870C0
:103A70009972D9721973997319745A619A61197785
:103A80001A625A621A859A8501321A708021C90019
:103A90009980654959855A73674D654C10AA6749E5
:103AA0002800A0470028F9D1634B1A68D37B5BB28A
:103AB000002BFBDB138802210B4313805E4B1A683B
:103AC000D37B5BB2002BFBDB80235371574C02226C
:103AD0005B4920005B4B9B46984720685A4B9A46AF
:103AE00098475A4B99461B5C1F26334001252A00F4
:103AF0009A401300464A904613601027637E3B436A
:103B00006376236810225A734B4C022250492000DE
:103B1000D8472068D0474B461B5C1E40B540434603
:103B20001D60637E1F436776236810225A73494BDA
:103B30001B6A5B0529D52E4B1B78DBB2DA09002402
:103B4000002A04D15C09E401424A944664441F22DD
:103B5000134001259D40E5610A203F4B9847E561F0
:103B6000244B1B78DBB2DA090024002A04D15C095B
:103B7000E401384A944664441F22134001259D40C5
:103B8000E5610A20344B9847E5615020324B984755
:103B9000304B1C6A8023DB001C40304B1B78202BF1
:103BA00060D02E4B1B78402B5CD053222C4B1A70CC
:103BB0005EE010220E4B1A7001320E4B1A70BAE6FC
:103BC0001916000035150000A52500005902002037
:103BD000F9160000A4010020DC0100209C02002056
:103BE0007C020020D0010020A801002094020020C7
:103BF0001A020020580200200200160002001700DE
:103C000000140042E0010020BD020000890D000008
:103C100000E100E09D260000490400007D26000030
:103C200029240000CD2D000071020000B401002005
:103C300029080000003000426002002000340042E9
:103C40009D210000F9060000F107000088550000E2
:103C5000D921000000440041810100003802002009
:103C6000B0010020E822B94B1A706D3AB84B1A70B7
:103C7000B84B1A78D2B2D1090023002904D15309D4
:103C8000DB01B5498C4663441F21114001228A4063
:103C90009A61B24B1A78D2B2D1090023002904D11B
:103CA0005309DB01AC498C4663441F2111400122BA
:103CB0008A405A610120AA4B9847AA4B1A68D37BC5
:103CC0005BB2002BFBDB00231371D37B5BB2002BB9
:103CD000FBDB40235371002C00D1F0E09E4B80228F
:103CE000D2025A61802212035A6104225A61FC32C4
:103CF0009A61186A0005C00F0B23FF3AC8219A4C3D
:103D0000A047041E1BD0944B80229A618022D201CE
:103D10009A617F228E4B1A70944B98470220944BE5
:103D2000984700270123984601260023019300931A
:103D300000258D4B99468F4B9B46CA4615E0864B16
:103D400080225A618022D2015A61E2E701270CE009
:103D5000814B80225A618022D2015A6112E00220F6
:103D6000854B984714E0002F12D10B230122C82164
:103D70002000C847041EEBD0774B80229A61802236
:103D8000D2019A615B461B68022BECD9002FE6D06A
:103D90004046431E9841C0B2062300220521D04769
:103DA0008046002803D1754B1B789B075BD4701E9F
:103DB0008641F0B20923002205216B4EB047061E52
:103DC00003D16E4B1B785B0753D46D4B1B78002BD4
:103DD00007D101226A4B1A70684A137808218B4375
:103DE0001370681E8541E8B218230122C8215E4F76
:103DF000B84705000098431E9841C0B20123012234
:103E0000C821B847009002900198431E9841C0B263
:103E100019230122C821B8470190002D2FD0029B01
:103E2000002B30D0002832D0564B1B78002B8DD081
:103E30000023544A13704F4A1360534B1A7892066A
:103E4000920F1B781B079B0F9A4224DD4E4B1A786A
:103E50009206920F1B789B079B0F9A421BDD6F22E5
:103E60003B4B1A7023E0454A137802218B431370B1
:103E70009DE7424A137804218B431370A5E7002085
:103E8000424B9847D0E70120404B9847CCE702309F
:103E90003E4B9847C8E73C4B1A781207920F1B78A5
:103EA0009B079B0F9A4206DD6B22294B1A702F4B02
:103EB0009847002759E76322254B1A70F7E71FA997
:103EC0000120334B9847334B1B789B079B0F012BEB
:103ED00018D0304B1B789B079B0F022B0DD02E4B1D
:103EE0001B78202B0ED02C4B1B7800220292402BEB
:103EF00008D02A4B984600F0C8FE2E331FAAD35C88
:103F0000FF2BECD12648274B984701230293F0E77B
:103F10000022254B1A70104B08325A618022D201C0
:103F20005A610122164B1A70094B1B78532B41D052
:103F3000194B1B78202B39D0174B1B78402B35D0D1
:103F40005322034B1A70094B984733E04402002078
:103F5000B00100201A020020004400415802002055
:103F6000A12A00001C02002055240000352C00006E
:103F7000152200004002002071230000980200205A
:103F80001B0200209B0200203C020020F5280000BC
:103F9000F9160000DC010020380200205501000065
:103FA000B80B0000810100005D020020D14B1B789E
:103FB000002BC5D1D04B1B789B0603D5CE4B1B786D
:103FC0005B077BD501239946CC4FB24606230022DE
:103FD00019210120B84704000923002219210120DA
:103FE000B8470500C44B1B785B0700D5A0E0002C48
:103FF00007D04B46002B04D0029B002B00D1A2E03F
:104000001C00BF4B1B785B2B0ED0BE4B1B78202BAC
:1040100000D192E0BB4B1B78402B00D18DE05B229E
:10402000B74B1A70B84B9847B44D601E8441E0B24C
:10403000062300221921A84700240028F5D0AE4B02
:104040001B789B0604D5AC4B1B785B0700D4A6E01D
:10405000AE4B08229A61043A5A61FC329A61A94B2C
:104060001B78202B04D0A74B1B78402B00D0D9E025
:10407000A04B1B78002B00D0D4E0A44B8022D202AE
:104080005A61802212039A619D4B1B785B2B00D1F1
:104090000AE19C4B1B78202B00D100E1994B1B7847
:1040A000402B00D1FBE09A4B1B78002B00D0FBE0AB
:1040B0005B22934B1A70944B9847F5E0934D802305
:1040C0006B6110A901274F7000248C707E3B0B7030
:1040D0001B20904B984780231B056B6120008E4B63
:1040E000984772B6BFF35F8F8C4D2C7020008C4BBD
:1040F000984707208B4B98472F70BFF35F8F62B6AE
:10410000894B98477E4B1B781B079B0FBB4200D106
:1041100058E7864B1B68DA7B52B2002AFBDB002291
:104120001A71DA7B52B2002AFBDB40225A7149E74E
:104130007F4B1B78DBB2994659E76E4B1B78002BFF
:1041400000D171E76BE7002D00D03FE70120794BEC
:1041500098476A4E784B9B4602E0009B002B17D194
:104160000923002219210020B04700905B461B68FC
:10417000042BF2D95346002BEFD15F33604A137002
:10418000614B98470122624B1A70A2462500E4E772
:104190000120614B9847002D00D117E74FE7002021
:1041A0005D4B984772B6BFF35F8F00225B4B1A706E
:1041B000624B98470720624B98470720614B98470E
:1041C000002804D15F4C0720A0470028FBD0012025
:1041D000534B9847544B98470122504B1A70BFF3EA
:1041E0005F8F62B6464B1B781B079B0F93420DD027
:1041F0004E4B1B68DA7B52B2002AFBDB00221A719D
:10420000DA7B52B2002AFBDB40225A7180223F4BFC
:104210005A6110A900230B708B704B701B203D4B13
:10422000984715E73A4B1B78002B30D0374B80224C
:10423000D2029A61802212035A61FE22424B1A7006
:104240000120424B984710AC21000020404B98477A
:104250002278294B1A70E27C3E4BDA70A27C9A706D
:10426000627C5A70227C1A70E27D3B4BDA70A27D30
:104270009A70627D5A70227D1A70E27E374BDA7036
:10428000A27E9A70627E5A70227E1A70FCE61F4BE4
:104290008022D2025A61802212035A61F4E6154B41
:1042A0001B78002B00D0FEE6124B1B78002B02D1AE
:1042B0000122104B1A70164B1B78002B02D00022E3
:1042C000134B1A7001201B4B9847104B80225A61E8
:1042D0008022D2015A61184B1B68042B01D900F0CF
:1042E00066FD00240023994600260025034F124B4B
:1042F0009B4636E0AC010020DC0100205524000084
:10430000B001002038020020352C0000004400419C
:104310005D020020F9130000712300000800002056
:10432000652500008D1B0000150100001C02002007
:104330001B02002015220000D80100201D250000CE
:10434000E51A0000091C00005C020020A525000001
:10435000F91600007C020020D0010020A8010020F6
:104360000124631E9C41E0B20F230122C821B847FB
:1043700004006B1E9D41E8B218230122C821B847F2
:1043800005000090731E9E41F0B201230122C82156
:10439000B847060001904A46531E9A41D0B21923ED
:1043A0000122C821B8478146039059460B68042B67
:1043B00012D8002CD5D000990029D1D0019B002B18
:1043C00007D0002801D000F00BFD012401260125B3
:1043D000C7E701240125C4E70120D54B9847D54BF9
:1043E0001B68042B01D800F0E9FCD34A137838216C
:1043F0008B4320210B431370009B002B01D100F055
:10440000D2FC019B002B0BD0039B002B0DD0002C6A
:1044100001D000F03AFC0320C84B984700F035FC6F
:104420000120C64B984700F030FC0220C34B984750
:1044300000F02BFC10AC21000120C14B9847FF225B
:104440003023E25421000120BE4B9847BE4B9847D1
:1044500000F0C2FC332704230122C8210020A0471A
:1044600000287ED10A30C047013F002FF3D14B46D0
:10447000002B03D1002E01D000F0DEFC5B46002BA8
:1044800001D100F0BDFC0A9B002B04D10B9B002B3B
:1044900001D000F0C2FCA84A137807218B43012108
:1044A0000B431370012200210020A84B9847009075
:1044B0000327A74B1B789B070BD4A64B8022D20265
:1044C0005A61802212035A61A14A137802210B43D8
:1044D000137009230022052101209F4EB047814619
:1044E0009E4B1B781B0748D40125994B1B78DB0793
:1044F0004ED44B46002B00D110E1002D63D101209A
:10450000974B9847039D944B99468A4F5326062311
:10451000002205210020C84704003B68042B02D973
:10452000002D00D1A9E1002CF1D00120804B98474B
:1045300081490B78382293431A00102313430B70E0
:104540007C4B1B68042B00D8CEE10B7838229343B8
:104550001A00182313430B700AE033277BE7332735
:1045600079E7754A137838218B4308210B43137080
:1045700001237C4A13700093BDE12800451EA84129
:10458000C0B2062300220521734DA8470500ACE701
:10459000744B1B78DBB24A46002A00D1BEE0002BE8
:1045A000ABD1714A1368022BFCD9634A13780721F7
:1045B0008B4305210B431370002200210020634B25
:1045C000984700900327624B1B78DB0600D45AE122
:1045D000624B1B78DB0600D479E15D4B1B781B072F
:1045E0009B0F032B24D0544A137807218B430121BE
:1045F0000B4313705C4A1368022BFCD9544B1B7895
:104600001B079B0F012B00D1FFE1514B1B781B07B0
:104610009B0F022B00D100E20022002100204B4B17
:104620009847009003274A4A13780C210B431370D4
:104630004D4B1B68022B08D94C4B1B78002B04D028
:10464000434B1B785B0600D5EFE1494B1B889BB2BF
:10465000454A1268934208D8434B1B68022B04D981
:104660003B4B1B785B0600D4E3E1009B012B00D1A0
:1046700015E20298431E9841C0B20F230122C821BF
:10468000354EB04702900990049A531E9A41D0B219
:1046900018230122C821304EB04704908346524669
:1046A000531E9A41D0B201230122C8212A4EB0479D
:1046B00082468146059A531E9A41D0B2192301229F
:1046C000C821254EB047059008900A90069A531EBF
:1046D0009A41D0B21C230122C8211F4EB047069038
:1046E0000B90079A531E9A41D0B21B230122C82176
:1046F000194EB047079006005346002B00D1A9E69B
:104700005B46002B00D128E7089B002B00D126E751
:10471000099B002B00D0CCE633279CE60120104BF0
:104720009847039A0092034B994617003DE0C04614
:1047300071230000D801002044020020F528000069
:10474000F91600009117000061170000D531000034
:104750005C0200200044004155240000DC010020E0
:10476000152200001B02002040020020A5010020AD
:1047700018020020CE4B1B68132B0ED9CD4B1B7893
:104780007B2B0AD0CB4B1B789B09022B05D07B22BD
:10479000C84B1A70C84B9847019F09230022052176
:1047A0000020C64EB04700282BD14B461B68042B77
:1047B00010D8009B002B0DD1BE4B1B785B2B09D072
:1047C000BC4B1B789B09022B04D05B22B94B1A709F
:1047D000B94B9847B64B1B68042BCBD9002FC9D1D6
:1047E000B44B1B785F2BC5D0B24B1B789B09022BB7
:1047F000C0D05F22AF4B1A70AF4B9847019B00931C
:10480000B8E70120AE4B9847AE4A1368022BFCD99B
:10481000A74B1B68132B12D8A54B1B68042B1DD963
:10482000A94A137807218B4303210B4313700022FD
:1048300001210020A54B984700900127C3E6A24A1A
:10484000137807218B4304210B43137000220021AE
:1048500001209E4B984700900227B4E69A4A1378AD
:1048600007218B4302210B431370002200210020FB
:10487000964B984700900327A5E68E4B1E708E4BF3
:104880009847019D4FE6904B1A7807218A43110003
:1048900006220A431A701A7838218A4311003022FE
:1048A0000A431A708A4B197810220A431A701B782F
:1048B0009B0604D4864A137840218B43137001224F
:1048C000844B1A70019B02930423009316E17E49E6
:1048D0000B78382293431A00082313430B707E4A47
:1048E000117810230B43137001227A4B1A70009B2E
:1048F000042B00D100E1FF22784B1A70744B1A7818
:1049000040210A431A701A7820210A431A706E4A0D
:10491000137807218B431370039B0293009B012B99
:1049200000D0EBE00320664B9847614B1B68312BAE
:1049300009D9654A137838218B4320210B43137022
:104940000122674B9A61664B8022D2015A6108228C
:104950005A614B32574B1A70574B98475E4B1B7836
:104960009B079B0F022B10D1009B042B0DD010AC8A
:10497000210001205B4B984700223023E2542100A4
:104980000120594B9847594B98470126012401258E
:104990004A4F6B1E9D41E8B218230122C821B84737
:1049A0000500601E8441E0B201230122C821B847FE
:1049B0000400731E9E41F0B219230122C821B8479A
:1049C0000600002CE5D1002DE3D10028E1D1002222
:1049D000474B1A700230474B98470120394E374DEC
:1049E0003D4C3368032B00D910E10623002205213A
:1049F000A84703002278520700D5FFE00120002BD2
:104A0000EFD1019B02930020EBE70022012100205F
:104A10002E4B98470090012705E600220021012037
:104A20002A4B984700900227FDE50220244B984727
:104A30001BE60220224B9847284B1B78DBB2FC2B4D
:104A400020D9214A137807210B431370022F12D06B
:104A5000032F09D0012F00D007E60022012110000A
:104A60001A4B9847009000E6002211001000174BE7
:104A700098470090F9E5002211000120134B984758
:104A80000090F2E5124B1A7840210A431A701A7806
:104A900020210A431A700122114B9A61E5E50A4967
:104AA0000B78382293431A00202313430B705FE5E1
:104AB000D8010020B0010020352C00005524000052
:104AC000712300004002002044020020D531000084
:104AD0005C0200201B020020DC010020A402002058
:104AE00000440041F9160000911700006117000012
:104AF000DD01002015220000019B0293D64C042505
:104B0000E5613220D54B9847E5610320D44B9847A7
:104B1000039B05931D000124002304930133069396
:104B2000D04B994629E00220CD4B9847CE4B1B68CD
:104B3000002B50D1019D0AE00220C94B9847039DEC
:104B4000C54E0427F7613220C44B9847F761C64B26
:104B50001B68042B02D9059B002B3ED0C24B1B685F
:104B6000042B01D9002D40D05B46002B05D05346C5
:104B7000002B00D1D6E6012304934B461B68312B52
:104B800000D9CFE60698431E9841C0B20F230122F8
:104B9000C821B64EB047069082460498431E9841FD
:104BA000C0B204230122C821B04EB047049083460E
:104BB0002000441EA041C0B2062300220521AB4CB8
:104BC000A047041E00D06FE1002DACD0A64B1B689F
:104BD000002BB5D1BBE7019DB2E75322A44B1A705D
:104BE000A44B9847019B0593B8E7A3490B7838225B
:104BF00093431A00182313430B7093E69F4A1278CD
:104C0000002A00D0FAE6019A0292F7E602209C4BB5
:104C100098473AE0904B08225A618022D2015A61AB
:104C200080225A61974B1B78DBB2DA090024002AF4
:104C300004D15C09E401884A944664441F2213406D
:104C400001259D40E5610A20844B9847E5618E4B24
:104C50001B78BF2B48D88C4B1B789B069B0F022BD5
:104C600042DC894B1B781B079B0F022B3CDC864BDD
:104C70001B789B079B0F022B36DC0022834B1A709C
:104C80008348764B984701230293824B1B78002B75
:104C900006D17E4B1E78F6B2002E01D1FFF738F90F
:104CA0007C4B1B78DBB20193002BB3D0774B1B7886
:104CB000DBB20393002BADD1774A13780124A343D1
:104CC00013700220664B98476C4B1C70032503231E
:104CD0000093023B0793069305939A46049302932D
:104CE000624C2F005546C4E4674B1A7892091B7832
:104CF0009B069B0F9A4219DD634B1A7892091B7829
:104D00001B079B0F9A4211DD5F4B1A7892091B78A3
:104D10009B079B0F9A4209DD6722554B1A70554B32
:104D200098470124514E4C4F5C4D28E0564B1A7861
:104D30009206920F1B781B079B0F9A420CDD524B79
:104D40001A789206920F1B789B079B0F9A4203DDFD
:104D50006F22474B1A70E2E74B4B1A781207920FFB
:104D60001B789B079B0F9A4203DD6B22404B1A7006
:104D7000D5E763223E4B1A70D1E76420A847601E36
:104D80008441E0B2092300220521B047041EF4D17A
:104D90000823BB61F1E738490B78382293431A00A6
:104DA000202313430B7000203D4B98476DE70120F3
:104DB000334B98472B4B1B68042BECD8264B802297
:104DC0009A618022D2019A61364B1B789B079B0F18
:104DD000022B01D1FFF72EFB01222E4B1A7054E754
:104DE0000120274B98471F4B1B68042BE6D922490B
:104DF0000B78382293431A00202313430B7044E7A7
:104E00001D490B78382293431A00202313430B705B
:104E10000020234B9847FFF7ABFB174A1378382144
:104E20008B4320210B4313704B46002B0FD00220E5
:104E30001B4B9847FFF79CFB5F460F490B783822C6
:104E400093431A00202313430B70002FE0D001205E
:104E5000134B9847FFF78CFB004400418101000091
:104E600015220000D8010020400200205524000037
:104E7000B0010020352C0000440200201B0200205D
:104E8000712300001A0200203C0200209B02002037
:104E9000B80B0000DD0100205C020020550100007D
:104EA000F5280000DC010020034B1B68002B00D01C
:104EB00042E6039D4BE6C046400200200022430824
:104EC0008B4274D303098B425FD3030A8B4244D3D2
:104ED000030B8B4228D3030C8B420DD3FF22090214
:104EE00012BA030C8B4202D31212090265D0030BD3
:104EF0008B4219D300E0090AC30B8B4201D3CB03C9
:104F0000C01A5241830B8B4201D38B03C01A52410A
:104F1000430B8B4201D34B03C01A5241030B8B420C
:104F200001D30B03C01A5241C30A8B4201D3CB02F7
:104F3000C01A5241830A8B4201D38B02C01A5241DC
:104F4000430A8B4201D34B02C01A5241030A8B42DF
:104F500001D30B02C01A5241CDD2C3098B4201D3F7
:104F6000CB01C01A524183098B4201D38B01C01A75
:104F7000524143098B4201D34B01C01A52410309EC
:104F80008B4201D30B01C01A5241C3088B4201D39B
:104F9000CB00C01A524183088B4201D38B00C01A48
:104FA000524143088B4201D34B00C01A5241411A6F
:104FB00000D20146524110467047FFE701B500207C
:104FC00000F006F802BDC0460029F7D076E770472A
:104FD0007047C04670B500260C4D0D4C641BA410E4
:104FE000A64209D1002600F0D1FA0A4D0A4C641BF2
:104FF000A410A64205D170BDB300EB589847013606
:10500000EEE7B300EB5898470136F2E798550000F9
:1050100098550000985500009C550000002310B5DD
:105020009A4200D110BDCC5CC4540133F8E70300B0
:105030008218934200D1704719700133F9E70000DC
:10504000002C0042003000420034004200080042C0
:10505000000C00420010004200140042B00F00009B
:10506000B00F00008C0F0000B00F00008C0F00008C
:10507000720F0000720F0000B00F0000B00F0000B0
:10508000B00F0000B00F0000B00F0000B00F000024
:10509000B00F0000B00F0000B00F0000B00F000014
:1050A000B00F0000B00F0000B00F0000B00F000004
:1050B000B00F0000B00F0000B00F0000B00F0000F4
:1050C000B00F00008C0F0000B00F00008C0F00002C
:1050D000B00F0000B00F0000B00F0000B00F0000D4
:1050E000B00F0000B00F0000B00F0000B00F0000C4
:1050F000B00F0000B00F0000B00F0000B00F0000B4
:10510000B00F0000B00F0000B00F0000B00F0000A3
:10511000B00F0000B00F0000B00F0000B00F000093
:10512000B00F0000B00F0000B00F0000B00F000083
:10513000B00F0000B00F0000B00F0000B00F000073
:10514000B00F0000B00F0000B00F0000B00F000063
:10515000B00F0000B00F0000B00F00008C0F000077
:105160008C0F0000940F0000940F0000940F0000BB
:10517000940F0000454574414D4F52502E756D45BA
:10518000AA190000A6190000A6190000081A0000BC
:10519000081A0000BE190000B0190000C419000070
:1051A000F6190000101B0000F01A0000F01A0000B1
:1051B0007C1B0000021B00001E1B0000F41A0000F4
:1051C0002C1B00006C1B0000B41B0000F61B000031
:1051D000F61B0000F61B0000A61B0000C21B00000F
:1051E000981B0000D01B0000E61B00003C1C0000C8
:1051F000181C0000181C00004E1C0000141C0000AD
:105200001C1C0000381C0000201C0000241C000096
:10521000B8260000CC260000D8260000E4260000B6
:10522000F0260000FC26000008270000B22700003E
:10523000B2270000B2270000B227000014270000A8
:1052400020270000B2270000B2270000B22700008C
:105250002C270000B2270000B2270000B227000070
:1052600038270000B2270000B2270000B227000054
:1052700044270000B2270000B2270000B227000038
:1052800050270000B2270000B2270000B22700001C
:10529000B2270000B2270000B2270000B2270000AA
:1052A000B2270000B2270000B2270000B22700009A
:1052B0005C270000B227000068270000B22700002A
:1052C000B2270000B2270000B2270000B22700007A
:1052D000B2270000B2270000B2270000B22700006A
:1052E000B2270000B2270000B2270000B22700005A
:1052F000B2270000B2270000B2270000B22700004A
:10530000B2270000B2270000B2270000B227000039
:10531000B2270000B2270000B2270000B227000029
:10532000B2270000B2270000B2270000B227000019
:10533000B2270000B2270000B2270000B227000009
:10534000B2270000B2270000B2270000B2270000F9
:10535000B2270000B2270000B2270000B2270000E9
:10536000B2270000B2270000B2270000B2270000D9
:10537000B2270000B2270000B2270000B2270000C9
:10538000B2270000B2270000B2270000B2270000B9
:1053900074270000B2270000B2270000B2270000E7
:1053A000B2270000B2270000B2270000B227000099
:1053B000B2270000B2270000B2270000B227000089
:1053C000B2270000B2270000B2270000B227000079
:1053D000B2270000B2270000B2270000B227000069
:1053E000B2270000B2270000B2270000B227000059
:1053F000B2270000B2270000B2270000B227000049
:10540000B2270000B2270000B2270000B227000038
:10541000B2270000B2270000B2270000B227000028
:10542000B2270000B2270000B2270000B227000018
:10543000B2270000B2270000B2270000B227000008
:10544000B2270000B2270000B2270000B2270000F8
:10545000B2270000B2270000B2270000B2270000E8
:10546000B2270000B2270000B2270000B2270000D8
:10547000B2270000B2270000B2270000B2270000C8
:10548000B2270000B2270000B2270000B2270000B8
:1054900082270000B2270000B2270000B2270000D8
:1054A000B2270000B2270000B2270000B227000098
:1054B000B2270000B2270000B2270000B227000088
:1054C000B2270000B2270000B2270000B227000078
:1054D0008E2700009A270000B2270000B2270000A4
:1054E000A6270000322E0000202F0000D42E00003E
:1054F0003C2F0000562F0000D22F0000D42E0000B9
:10550000D42E0000D42E0000D42E0000D42E000093
:1055100000300000D42E0000D42E0000D42E000055
:10552000D42E000028300000D42E0000D42E00001D
:10553000D42E00007A300000D42E0000D42E0000BB
:10554000D42E000028310000D42E0000D42E0000FC
:10555000D42E0000D42E0000D42E0000D42E000043
:10556000D42E0000D42E0000D42E0000D42E000033
:10557000D42E0000D42E0000D42E0000D42E000023
:10558000D42E00007A31000012131400F8B5C04682
:10559000F8BC08BC9E467047DD000000F8B5C04668
:0C55A000F8BC08BC9E467047B500000037
:1055AC00401F00000800000001000000504D435F48
:0855BC0055430004060600003F
:04000003000020B920
:00000001FF
